:020000040800F2
:1000000000070020E5040008B915000839150008AC
:10001000911500083915000865150008E704000867
:10002000E7040008E7040008E7040008993700081F
:10003000E7040008E7040008E7040008E7040008F4
:10004000E7040008E7040008E7040008E7040008E4
:10005000E7040008E7040008C53B0008F13B00087E
:100060001D3C0008493C0008753C0008E7040008F6
:10007000E7040008E7040008E7040008E7040008B4
:10008000E7040008E7040008E704000871250008F9
:10009000DD2500083126000885260008A13C00085F
:1000A000E7040008E7040008E7040008E704000884
:1000B000153A0008E7040008E7040008E704000810
:1000C000E7040008E7040008E7040008E704000864
:1000D000E7040008E70400081D290008E7040008F9
:1000E000093D0008E7040008E7040008E7040008E9
:1000F000E7040008E7040008E7040008E704000834
:10010000E7040008E7040008E7040008E704000823
:10011000E7040008E7040008E7040008E704000813
:10012000E7040008E7040008E7040008E704000803
:10013000E7040008E7040008E7040008E7040008F3
:10014000E7040008E7040008E7040008E7040008E3
:10015000E7040008E7040008E7040008E7040008D3
:10016000E7040008E7040008E7040008E7040008C3
:10017000E7040008E7040008E7040008E7040008B3
:10018000E7040008E7040008E7040008E7040008A3
:10019000E7040008E7040008E7040008E704000893
:1001A000E7040008E7040008E7040008E704000883
:1001B000E7040008E7040008E7040008E704000873
:1001C000E7040008E7040008E7040008E704000863
:1001D000E7040008E7040008E7040008E704000853
:1001E00053B94AB9002908BF00281CBF4FF0FF319E
:1001F0004FF0FF3000F074B9ADF1080C6DE904CE9A
:1002000000F006F8DDF804E0DDE9022304B07047F1
:100210002DE9F047089D04468E46002B4DD18A42B9
:10022000944669D9B2FA82F252B101FA02F3C2F1EC
:10023000200120FA01F10CFA02FC41EA030E94407D
:100240004FEA1C48210CBEFBF8F61FFA8CF708FB9E
:1002500016E341EA034306FB07F199420AD91CEB76
:10026000030306F1FF3080F01F81994240F21C81A8
:10027000023E63445B1AA4B2B3FBF8F008FB1033F0
:1002800044EA034400FB07F7A7420AD91CEB040425
:1002900000F1FF3380F00A81A74240F207816444F5
:1002A000023840EA0640E41B00261DB1D44000237A
:1002B000C5E900433146BDE8F0878B4209D9002DDE
:1002C00000F0EF800026C5E9000130463146BDE868
:1002D000F087B3FA83F6002E4AD18B4202D38242D2
:1002E00000F2F980841A61EB030301209E46002D81
:1002F000E0D0C5E9004EDDE702B9FFDEB2FA82F2D6
:10030000002A40F09280A1EB0C014FEA1C471FFA33
:100310008CFE0126200CB1FBF7F307FB131140EA1A
:1003200001410EFB03F0884208D91CEB010103F1E7
:10033000FF3802D2884200F2CB804346091AA4B2A9
:10034000B1FBF7F007FB101144EA01440EFB00FE7D
:10035000A64508D91CEB040400F1FF3102D2A645E2
:1003600000F2BB800846A4EB0E0440EA03409CE781
:10037000C6F12007B34022FA07FC4CEA030C20FA2E
:1003800007F401FA06F31C43F9404FEA1C4900FA4E
:1003900006F3B1FBF9F8200C1FFA8CFE09FB1811CB
:1003A00040EA014108FB0EF0884202FA06F20BD93E
:1003B0001CEB010108F1FF3A80F08880884240F28E
:1003C0008580A8F102086144091AA4B2B1FBF9F0D2
:1003D00009FB101144EA014100FB0EFE8E4508D9CD
:1003E0001CEB010100F1FF346CD28E456AD9023852
:1003F000614440EA0840A0FB0294A1EB0E01A14237
:10040000C846A64656D353D05DB1B3EB080261EBA4
:100410000E0101FA07F722FA06F3F1401F43C5E97E
:10042000007100263146BDE8F087C2F12003D840B4
:100430000CFA02FC21FA03F3914001434FEA1C47F6
:100440001FFA8CFEB3FBF7F007FB10360B0C43EAE8
:10045000064300FB0EF69E4204FA02F408D91CEB98
:10046000030300F1FF382FD29E422DD90238634496
:100470009B1B89B2B3FBF7F607FB163341EA034136
:1004800006FB0EF38B4208D91CEB010106F1FF3885
:1004900016D28B4214D9023E6144C91A46EA00467C
:1004A00038E72E46284605E70646E3E61846F8E60E
:1004B0004B45A9D2B9EB020864EB0C0E0138A3E757
:1004C0004646EAE7204694E74046D1E7D0467BE738
:1004D000023B614432E7304609E76444023842E7B0
:1004E000704700BF02E000F000F8FEE772B63A483D
:1004F00080F30888394880F3098839484EF6085156
:10050000CEF20001086040F20000CCF200004EF68E
:100510003471CEF200010860BFF34F8FBFF36F8FCD
:1005200040F20000C0F2F0004EF68851CEF2000119
:100530000860BFF34F8FBFF36F8F4FF00000E1EE05
:10054000100A4EF63C71CEF200010860062080F3DE
:100550001488BFF36F8F03F09FF903F07BF903F06A
:10056000C5F94FF055301F491B4A91423CBF41F835
:10057000040BFAE71C49194A91423CBF41F8040BAD
:10058000FAE71A491A4A1B4B9A423EBF51F8040B2C
:1005900042F8040BF8E700201749184A91423CBF83
:1005A00041F8040BFAE703F059F903F0EDF9144CA4
:1005B000144DAC4203DA54F8041B8847F9E700F005
:1005C00041F8114C114DAC4203DA54F8041B884732
:1005D000F9E703F041B900000007002000230020E4
:1005E00000000008000100200007002078400008FB
:1005F00000230020242300202823002098390020F5
:10060000E0010008E0010008E0010008E001000846
:100610002DE9F04F2DED108AC1F80CD0C3689D462E
:10062000BDEC108ABDE8F08F002383F311882846C3
:10063000A047002002F086FDFEE702F00BFD00DF80
:10064000FEE700002DE9F04103F044F8074603F00F
:100650008FF8054600283DD12B4B9F423AD00133FD
:100660009F423AD0294B27F0FF029A4239D1F8B283
:1006700000F052FAA84642F2107400F055FC08B19E
:100680000024A04600F04EFA064670B37CBB4646F6
:1006900035B11F4B9F4203D003F062F80024264679
:1006A000002003F021F81B4B1B691B0422D40EB160
:1006B00000F032F800F096FC00F07CFE00F07EFFC7
:1006C0000546CCB100F07AFF401BA04214D900F0DF
:1006D00023F8F3E7A8460024CFE704464FF00108CB
:1006E000CBE780464FF47A74C7E70446D0E74FF46F
:1006F0007A74CDE70024DDE700F026FD4FF47A7030
:1007000002F026FDDDE700BF010007B0000008B0E1
:10071000263A09B0000402401E4B1F4A10B51C4681
:100720001968013134D004339342F9D162681B4B0C
:100730009A422DD91A4B9B6803F1006303F580336D
:100740009A4225D202F0E0FF02F0F2FF002000F012
:100750004BFE144B0220187000F082FE124B1A6CF4
:1007600000221A64196E1A66196E596C5A64596E11
:100770005A665B6E72B64FF0E0232021C3F8084D35
:10078000D4E9003281F311889D4683F3088810472D
:1007900010BD00BF0000010820000108FFFF000895
:1007A000002300202823002000380240094A136853
:1007B00049F2690099B21B0C00FB01331360064B30
:1007C000186844F2506182B2000C01FB020018600C
:1007D00080B27047202300201C23002010B5002188
:1007E0001022044600F058FE034B03CB20606160EA
:1007F0001868A06010BD00BF107AFF1F2DE9F043FC
:10080000224DBBB000F0DAFEAB6840F2ED22C31A15
:10081000934232D906AFA8602B46282200213846E1
:1008200001F0DAFB05F10E0000F02EFE0026044672
:100830005FFA80F905F10E08F3B2F100994501F174
:10084000280107D908EB06030822384601F0C4FB4B
:100850000136F1E708230122CDE9023205340C4BC1
:100860000193A4B230230093CDE9047405A3D3E926
:100870000023297B074801F0C7F93BB0BDE8F083AE
:10088000AFF3008078F6339F93CACD8D703300208C
:100890007D3300204433002070B50D4614461E46BB
:1008A00001F048F950B9022E10D1012C0ED112A33B
:1008B000D3E90023C5E90023012007E0282C10D04C
:1008C00005D8012C09D0052C0FD0002070BD302C8C
:1008D000FBD10BA3D3E90023ECE70BA3D3E900235F
:1008E000E8E70BA3D3E90023E4E70BA3D3E9002354
:1008F000E0E700BFAFF30080401DA12026812A0B56
:1009000078F6339F93CACD8D9E6AC421818A46EEC4
:1009100026417272DF25D7B7F017304A39059E5647
:1009200013B504462346084620220021019001F019
:1009300053FB22790198032A234628BF032203F898
:10094000042F2021022201F047FB62790198072A37
:10095000234628BF072203F8052F2221032201F096
:100960003BFBA2790198072A234628BF072203F8F8
:10097000062F2521032201F02FFB019804F1080323
:100980001022282101F028FB382002B010BD000001
:100990002DE9F04FFFB01FAD0CAE40F2751280464E
:1009A0000F4620A80021296000F076FD4822002192
:1009B000304600F071FD00F001FE554B4FF47A72A5
:1009C000B0FBF2F0186093E80700012386E8070007
:1009D0000DF152003382FFF701FF4FF4A24333843D
:1009E00006AB18464B4903F039FA15223064294604
:1009F000304686F83C20FFF793FF10AB04460146D3
:100A00000822284601F0E8FA0822A1180DF1410356
:100A1000284601F0E1FA0DF14203082204F1100129
:100A2000284601F0D9FA11AB202204F1180128461A
:100A300001F0D2FA12AB402204F13801284601F04D
:100A4000CBFA14AB082204F17801284601F0C4FA6D
:100A50000DF15103082204F18001284601F0BCFA8F
:100A600004F1880A0DF1520904F5847B4B46514686
:100A7000082228460AF1080A01F0AEFAD34509F126
:100A80000109F3D119AB08225946284601F0A4FA0E
:100A900004F588744FF0000996F834304B450AD9B4
:100AA000B36B21464B440822284601F095FA0834DE
:100AB00009F10109F0E74FF0000996F83C304B4589
:100AC00004EBC90108D9336C08224B44284601F0D5
:100AD00083FA09F10109F0E700230393BB7E029337
:100AE000073107F119030193C1F3CF010123CDE9C8
:100AF00004510093F97E04A3D3E90023404601F09A
:100B000083F87FB0BDE8F08F9E6AC421818A46EEEB
:100B10002C2300206C3E0008014B1870704700BF6A
:100B200038230020F0B5324B1C7B85B034B1314BFB
:100B30000E221A810024204605B0F0BD2E4A10680E
:100B4000516802AB03C308232C492D480DEB030267
:100B500003F062F9054630B9264B2A480A221A8169
:100B600000F0E6FCE6E70169B1F5E02F06D9214B7C
:100B700025480B221A8100F0DBFCDCE7438B512B6C
:100B800008D01C4A21480C2111815122194600F03D
:100B9000CFFCD0E71E4A024402F11003994204D26E
:100BA000144B1C4810221A81E5E710398E1A204692
:100BB000134900F007FD3246074605F118012046AB
:100BC00000F000FDAB689F4202D1EB6898420AD06A
:100BD000084B0D221A810090D5E902123B460E48BF
:100BE00000F0A6FCA6E70D4800F0A2FC0124A2E755
:100BF000703300202C230020153F0008DCFF060086
:100C000000000108843E0008903E0008A23E000853
:100C10000800FFF7C03E0008DD3E0008063F000860
:100C20002DE9F04FADB006AF80460C4600F082FFD4
:100C3000054600285AD1237E022B1BD1E38A012BC3
:100C400018D100F0BBFC0646FFF7B0FD03464FF499
:100C5000C870DFF8D092B3FBF0F206F5167602FB0F
:100C6000103316FA83F3C9F80030E37E33B9A84B8A
:100C700000221A709C37BD46BDE8F08FA38AEEB201
:100C8000013BB34205F101050BD93B1D1E44E900B0
:100C900000960023082201F0F801204601F060F8D8
:100CA000ECE707F11400FFF799FD324607F1140154
:100CB000381D03F0A1F80028D9D10F2E08D8944B85
:100CC0001E70D9F80030A3F51673C9F80030D1E7CB
:100CD000FB1CF8700146009307220346204601F0F2
:100CE0003FF8F978404600F01DFFC3E7E38A282B60
:100CF00026D010D8012B1ED0052BBBD1BFF34F8FB0
:100D00008449854BCA6802F4E0621343CB60BFF3A9
:100D10004F8F00BFFDE7302BACD1637E7F4D013399
:100D20006A7BDBB29342E94603D1E27E2B7B9A4297
:100D300065D0CD469EE721464046FFF729FE99E75C
:100D4000A38A013B9BB2C92B94D8744D2E7B26BB42
:100D500005F10C030093082233463146204600F08B
:100D6000FFFF731CF2B2D9001E46A38A013B9A42D0
:100D700005DA0E322A44009200230822EEE700230F
:100D80000022C5E900230023AB6085F8D730C5F801
:100D9000D8302B7B0BB9E37E2B73002507F11409A8
:100DA0003B1D082229464846C7E90155FD6001F070
:100DB00013F93B7A05F1010AAB424FEACA0608D99A
:100DC000FB6808222B443146484601F005F9554698
:100DD000EFE7C6F3CF06E17ECDE904960023039347
:100DE000A37E0293193428230093019446A3D3E9E8
:100DF0000023404600F008FFFFF700FD3AE74FF000
:100E0000000807F11403A7F814801022009341464C
:100E10000123204600F0A4FFA68A023EB6B2F31CCE
:100E20009B109B000733DB08A9EBC3039D460DF124
:100E3000180A1FFA88F34FEAC801B34201F1100102
:100E40000AD20AEB0803009308220023204600F090
:100E500087FF08F10108ECE795F8D70000F0CEFA1B
:100E6000D5F8D83004461BB995F8D70000F0D6FA6B
:100E7000D5F8D83033449C4204D295F8D7000130DD
:100E800000F0CCFA4FEA960B4FF000081FFA88F1F9
:100E90008B45D5E9003209D90AEB880103EB8800BC
:100EA000012200F001FB08F10108EFE7F31842F11D
:100EB0000002C5E90032D5F8D83095F8D70006EB26
:100EC0000308C5F8D88000F099FA804509D395F851
:100ED000D730D5F8D8000133001B85F8D730C5F8D6
:100EE000D800FF2E08D800232B7300F0A9FAFFF7D3
:100EF00019FE08B1FFF710FC2B68094A9B0A013361
:100F000013810023AB6014E726417272DF25D7B747
:100F10003D33002000ED00E00400FA0570330020AE
:100F20002C2300204033002030B54FF00054244BD8
:100F300022689A4285B007D002F024FC0446A8B982
:100F40000024204605B030BD1E4B627D1A701E483D
:100F5000237D03731D49C9220E3000F08BFA204611
:100F6000E022002100F098FA0124EAE7184A194D1E
:100F7000136C43F000731364AA6D174B9A42DFD1D0
:100F80002B6E013B7E2BDBD8144A07CA01AB83E8EA
:100F900007001846032100F02BFB6B6D83424FF0D6
:100FA0000003CDD12A6D8A4201BFAB65054B2A6E85
:100FB0001A7003BF0A4BEA6D1A601C46C1E700BFF6
:100FC0009AAD44C53823002070330020160000205D
:100FD00000380240006600405041A0B05866004012
:100FE000182300202DE9FF474B4C02236371002397
:100FF00002934A4BD3F800C0BCF57A7F12D3484B1A
:10100000484FB7FBFCF69C458CBF0A231123581EA2
:10101000B6FBF3F503FB1562C1B2002A3ED00228ED
:101020000346F4D89DF80B303F4940485A1E9DF8BE
:101030000A30013B1B0443EA0253BDF80820013A81
:1010400013434B6001F026FD00230193384B3949CF
:1010500000933948394B4FF4805200F03DFD384B36
:10106000197811B1344800F05DFD00F0A7FA05468B
:10107000FFF79CFB4FF4C873B0FBF3F202FB1303C2
:1010800005F5167010FA83F02E4B186002F070FB15
:1010900008B10F23238104B0BDE8F0876B1EB3F5C0
:1010A000806FBFD2C1EBC10E0EF103034FEAE3091B
:1010B000C3F3C703A1EB030809F1010A4FF47A70E7
:1010C0005FFA88F609FB00005AFA88F8B0FBF8F0DE
:1010D000B0F5617F08D90EF1FF33C3F3C703C91A16
:1010E000CEB2591E0F2914D8721E072A8CBF0022B7
:1010F0000122991901FB0551B7FBF1F7BC4591D1CC
:10110000002A8FD0ADF808508DF80A308DF80B60AA
:1011100088E71346EDE700BF2C23002018230020AA
:101120003F420F0040787D011023002088340020CA
:10113000990800083C23002044330020210C0008BB
:1011400038230020403300202DE9F04F91A7D7E944
:1011500000670FF24829D9E90089874D93B0DFF87D
:1011600044B2864C284600F0B3FD0DF1300A0790DA
:1011700070B310220021504600F08EF9079B197BB6
:101180004FF0000261F303028DF83020586899682F
:101190000EAA03C21B680D9A63F31C029DF830303F
:1011A0000D9243F020038DF830300023524619464B
:1011B000584601F07FFC079028B9284600F08CFDC6
:1011C000079B2370CEE72378072B3CD8013323708D
:1011D00018220021504600F05FF9DFF8C8B1684CD2
:1011E000002319465246584601F08CFC014670BB5C
:1011F000102208A800F050F9636983F480636361EA
:1012000000F0DEF90B4612A9024611E903000DF1C8
:10121000240C8CE803009DF83410C1F30300890608
:101220004CBF0E99BDF838C08DF82C0046BFC1F3F5
:101230001C0C4CF00041CCF30A010891284608A987
:1012400000F012FFCCE7284600F046FDC0E7284634
:1012500000F070FC0446002848D1DFF84CB100F0E3
:10126000ADF9DBF80030984240D300F0A7F90790C1
:10127000FFF79CFA079A8DF8204003464FF4C87098
:1012800002F51672B3FBF0F101FB103312FA83F38F
:10129000CBF80030DFF814B19BF8001011B901232E
:1012A0008DF8203050460791FFF798FA0799C1F161
:1012B0001004E4B2062C28BF0624224651440DF146
:1012C000210000F0D7F808AB0393182302930134F0
:1012D0002C4B0193E4B20123009304943B46324625
:1012E000284600F029FC00238BF8003000F066F956
:1012F000254A264C1368C31AB3F57A7F31D31060A0
:1013000000F05EF902460B46284600F0EFFC284646
:1013100000F010FC28B3237BDFF894B0002B14BF3F
:10132000032302238BF8053000F048F94FF47A7359
:101330005146B0FBF3F0CBF800005846FFF7F0FA47
:10134000182307300293124B0193C0F3CF0040F2F1
:101350005513CDE903A0009342464B46284600F0C2
:10136000EBFB237B2BB1FFF749FA237B002B7FF4A8
:10137000F6AE13B0BDE8F08F4433002055340020A2
:10138000000002403C330020503400207033002025
:1013900054340020401DA12026812A0BF1C6A7C18C
:1013A000D068080F88340020403300203D330020EF
:1013B0002C23002070B502F02DF8094E094D308025
:1013C000002428683388834208D902F01DF82B686E
:1013D00004440133B4F5803F2B60F2D370BD00BFED
:1013E000843400205834002002F0D8B800F10060A6
:1013F000920000F5803002F05BB80000054B1A68DF
:10140000054B1B889B1A834202D9104401F0FCBF94
:1014100000207047583400208434002038B5074D30
:1014200004462868204401F0F7FF28B928682044C2
:10143000BDE8384002F008B838BD00BF583400207D
:10144000064991F8243033B10023086A81F824302A
:101450000822FFF7CBBF0120704700BF5C3400209B
:10146000022802BF024B4FF480629A61704700BFAE
:101470000000024010B50023934203D0CC5CC4545A
:101480000133F9E710BD000003460246D01A12F9F5
:10149000011B0029FAD1704702440346934202D04F
:1014A00003F8011BFAE770472DE9F8431F4D144676
:1014B00095F824200746884652BBDFF870909CB30D
:1014C00095F824302BB92022FF2148462F62FFF7E0
:1014D000E3FF95F82400C0F10802A24228BF22468B
:1014E000D6B24146920005EB8000FFF7C3FF95F8A6
:1014F0002430A41B1E44F6B2082E17449044E4B2D4
:1015000085F82460DBD1FFF79BFF0028D7D108E0E6
:101510002B6A03EB82038342CFD0FFF791FF0028B1
:10152000CBD10020BDE8F8830120FBE75C3400202C
:101530000FB4002004B0704700B59BB0EFF30981F1
:1015400068226846FFF796FFEFF30583044B9A6B1A
:10155000DA6A9A6A9A6A9A6A9A6A9A6A9B6AFEE749
:1015600000ED00E000B59BB0EFF30981682268460A
:10157000FFF780FFEFF30583044B9A6B9A6A9A6A30
:101580009A6A9A6A9A6A9B6AFEE700BF00ED00E0D9
:1015900000B59BB0EFF3098168226846FFF76AFF48
:1015A000EFF30583034B5A6B9A6A9A6A9A6A9A6AAE
:1015B0009B6AFEE700ED00E0FEE7000002F028B8BD
:1015C00002F000B830B5094D0A4491420DD011F82F
:1015D000013B5840082340F30004013B2C4013F02A
:1015E000FF0384EA5000F6D1EFE730BD2083B8ED69
:1015F000F7B54FF0FF33DFF854C0DFF854E000EBED
:1016000081011A4688421CD050F8044B019401AF66
:10161000042417F8015B82EA05620825DB181646E8
:1016200005F1FF355241002EBCBF83EA0C0382EA6C
:101630000E0215F0FF05F1D1013C14F0FF04E8D1D2
:10164000E0E7D843D14303B0F0BD00BF9336EAA929
:10165000EBE1F0422DE9F041C56915B9C161BDE882
:10166000F0814B6823F06047C3F38A464FEAD37E8C
:10167000C3F3807816EA230638BF3E46AC462B46B5
:101680005A68BEEBD27F22F060440AD0002A18DAF2
:10169000A40CB44217D19D420FD10D60DEE7134672
:1016A000EEE7A74207D102F08044C2F380724245C0
:1016B0000BD054B1EFE708D2EDE7CCF800100B6087
:1016C000CDE7B44201D0B442E5D81A689C46002A5E
:1016D000E5D11960C3E700002DE9F047089D01F04E
:1016E00007044FEAD508224405F0070500EBD100B6
:1016F0004FF47F49944201D1BDE8F08704F0070719
:1017000005F0070A57453E4638BF5646C6F108065B
:10171000111B8E4228BF0E46E10808EBD50E415C36
:1017200013F80EC0B94029FA06F721FA0AF1FFB200
:101730008CEA010147FA0AF739408CEA010C03F8F8
:101740000EC034443544D5E780EA0120082341F235
:10175000210201B24000002980B203F1FF33B8BF7B
:10176000504013F0FF03F4D17047000038B50C4629
:101770008D18A54200D138BD14F8011BFFF7E4FF16
:10178000F7E7000002684AB113680360C388018963
:1017900001339BB29942C38038BF03811046704722
:1017A00070B588B0202204460D4668460021FFF738
:1017B00073FE20460495FFF7E5FF024658B16B46DD
:1017C000054608AE1C4603CCB44228606960234637
:1017D00005F10805F6D1104608B070BD082817D9E4
:1017E00009280CD00A280CD00B280CD00C280CD0BF
:1017F0000D280CD00E2814BF4020302070470C203C
:101800007047102070471420704718207047202020
:1018100070470000082817D90C280CD910280CD9BB
:1018200014280CD918280CD920280CD930288CBFA2
:101830000F200E207047092070470A2070470B20A8
:1018400070470C2070470D207047000010B54B68A2
:1018500023B9CA8A63F30902CA8210BDC4681A6830
:101860001C60C360438A013B43824A60EFE700008B
:101870002DE9F84F1D46CB8A0F46C3F3090106290F
:10188000814692460B4630D00020AAB207F11904D7
:101890009EB2052E1FFA80F80FD8904503F1010380
:1018A00006D3FB8A0A4462F30903FB8201201AE093
:1018B0001AF80060E6540130EAE79045F1D2A1F150
:1018C000060B1C237C68BBFBF3F203FB12BB1FFA65
:1018D0008BF6002C45D14846FFF754FF044638B933
:1018E00078606FF00200BDE8F88F4FF00008E6E77F
:1018F000002606607860ADB24FF0000B454510D968
:101900000AEB0803221D13F8011B9155B1B208F12F
:1019100001081B291FFA88F82BD0454506F101065E
:10192000F1D8FB8AC3F30902154465F30903BCE748
:10193000013292B21C462368002BF9D1AB1F0B4435
:101940001C21B3FBF1F301339BB29A42D3D2BBF11A
:10195000000FD0D14846FFF715FF20B9C4F800B0FA
:10196000BFE70122E7E7C0F800B05E46206004460A
:10197000C1E74545D5D94846FFF704FF08B92060BF
:10198000AFE7C0F800B0002620600446B6E70000CC
:101990002DE9F04F2DED028B83B0CDE90013BDF89A
:1019A0003C5007469146002A00F092802DB10E9BD4
:1019B000002B00F08D80072D32D807F10C00FFF7C7
:1019C000E1FE044638B96FF00204204603B0BDECD6
:1019D000028BBDE8F08F14220021FFF75DFD0E9908
:1019E0002A4604F10800FFF745FD681CC0B2FFF766
:1019F00011FFFFF7F3FE207499F80030013814FA54
:101A000080F003F01F0363F03F030372009B43F079
:101A10000041616038462146FFF71CFE0124D4E7EF
:101A200000F10C034FF0000808EE103A4FF0800A66
:101A30004646444618EE100AFFF7A4FE83460028E7
:101A4000C1D014220021FFF727FDC6BB019BABF8D4
:101A5000083002200E9B00F1080299195BFA82F20D
:101A60000130C0B2082801D0AE422AD3FFF7D2FE1F
:101A7000FFF7B4FE99F80020009B411E02F01F0200
:101A800042EA4812AE4208BF4FF0400A5BFA81F1C9
:101A90004AEA020A43F0004281F808A08BF81000DD
:101AA000CBF8042059463846FFF7D4FD0134AE4246
:101AB00024B288F001084FF0000ABBD185E700206E
:101AC000C8E711F801CB02F801CB0136B6B2C7E77F
:101AD0006FF0010479E70000F8B515460E4628229C
:101AE000002104461F46FFF7D7FC069B6360B5F54F
:101AF000001F079BA76034BF6A094FF6FF7223627D
:101B000004F10C0097B200239A4205D80023036029
:101B100027826382A382F8BD0660013330462036F7
:101B2000F2E7000003781BB94BB2002BC8BF01706D
:101B300070470000007870472DE9F74FDDF83C90C2
:101B4000BDF830500D9E9DF83840BDF8407080467D
:101B500092469B46B9F1000F01D1002F51D11F2CA5
:101B60004FD898F80000B0B9072F47D835F00303D5
:101B700047D13A4649464FF6FF70FFF7F7FD20F090
:101B800001002D02400445EA0464400C44EA40246C
:101B90004FF6FF7321E040EA0520072F40EA046476
:101BA000F6D900254FF6FF73C5F12000A5F12002FC
:101BB0002AFA05F10BFA00F001432BFA02F2114365
:101BC0001846C9B2FFF7C0FD0835402D0346EBD1DA
:101BD0003A464946FFF7CAFD0346CDE9009732462B
:101BE00021464046FFF7D4FE33780133DBB21F2B8A
:101BF00088BF0023337003B0BDE8F08F6FF003009F
:101C0000F9E76FF00100F6E72DE9F04F85B0924655
:101C1000DDF848800F9D9DF840209DF84490BDF868
:101C20004C7006469B46B8F1000F01D1002F48D1F9
:101C30001F2A46D83378002B46D00C0244EA0264AF
:101C40009DF8381044EAC93444EA01441C43072F84
:101C500044F0800432D900234FF6FF72C3F1200C08
:101C6000A3F120002AFA03F10BFA0CFC41EA0C0163
:101C70002BFA00F00143C9B210460393FFF764FD4D
:101C8000039B0833402B0246E8D13A464146FFF712
:101C90006DFD0346CDE900872A4621463046FFF711
:101CA00077FEB9F1010F06D12B780133DBB21F2B80
:101CB00088BF00232B7005B0BDE8F08F4FF6FF738F
:101CC000E8E76FF00100F6E76FF00300F3E70000CC
:101CD000C06900B104307047C3691A68C261C26844
:101CE0001A60C360438A013B438270472DE9F0418B
:101CF000D0F81880194E14461D464146002709B9F0
:101D0000BDE8F081D1E90223A21A65EB03039642F4
:101D100077EB03031ED283698B420DD1FFF796FD4B
:101D200083691B688361C3680B60438AC1608169F2
:101D3000013B43828846E2E7FFF788FD0B68C8F85D
:101D40000030C3680B60438AC160013B4382D8F80E
:101D50000010D4E788460968D1E700BF80841E00E0
:101D60002DE9F04F8BB00D46DDF8509014469B46A0
:101D70008046002800F01981B9F1000F00F01581AC
:101D8000531E3F2B00F21181012A03D1BBF1000F3A
:101D900040F00B810023CDE90833B8F81430B5EBDF
:101DA000C30F4FEAC30703D300200BB0BDE8F08F89
:101DB0002B199F42D8F80C303ABF7F1BFFB2274641
:101DC0001BB9D8F81030002B7AD02F2D4ED8C5F182
:101DD0003006B7424FF000032CBFF6B23E460093E8
:101DE0002946D8F8080008AB3246FFF775FCA7EB88
:101DF000060A35445FFA8AFAB8F8143003F1005342
:101E0000063BDB000493D8F80C3003933021039B8E
:101E100013B1BAF1000F2CD1D8F8100040B1BAF1CB
:101E2000000F05D0009608AB5246691AFFF754FC24
:101E300038B2002FB8D066070AD00AAB03EBD40142
:101E4000624211F8083C02F00702134101F8083C15
:101E5000082C3CD9102C40F2B580202C40F2B780E1
:101E6000BBF1000F00F09C80082334E0BA46002646
:101E7000C2E7049BE02B28BFE02306930B44AB4250
:101E8000059314D95A1B03980096924534BF5246C5
:101E9000D2B2691A08AB04300792FFF71DFC079A0B
:101EA0001644AAEB020A1544F6B25FFA8AFA049BBA
:101EB000069A05999B1A0493039B1B680393A6E754
:101EC0000093D8F8080008AB3A462946AEE7BBF1C4
:101ED000000F13D00123B4EBC30F6CD0082C12D821
:101EE0009DF82030621E23FA02F2D50706D54FF086
:101EF000FF3202FA04F423438DF820309DF820309D
:101F000089F8003051E7102C12D8BDF82030621E3D
:101F100023FA02F2D10706D54FF0FF3202FA04F499
:101F20002343ADF82030BDF82030A9F800303CE75D
:101F3000202C0FD80899631E21FA03F3DA0705D580
:101F40004FF0FF3202FA04F40C430894089BC9F8DE
:101F500000302AE7402C2BD0DDE90865611EC4F172
:101F60002102A4F1210326FA01F105FA02F225FA71
:101F700003F311431943CB0712D50122A4F1200327
:101F8000C4F1200102FA03F322FA01F1A240524205
:101F900043EA010363EB430332432B43CDE90823B8
:101FA000DDE90823C9E90023FFE66FF00100FCE644
:101FB0006FF00800F9E6082CA0D9102CB3D9202C1A
:101FC000EED8C3E7BBF1000FADD0022383E7BBF12E
:101FD000000FBBD004237EE730B5012A144638BF7A
:101FE0000124402C85B028BF40240025012ACDE9DA
:101FF000025518D81B788DF8083063070AD004AB57
:1020000003EBD405624215F8083C02F00702934046
:1020100005F8083C009103462246002102A8FFF77C
:102020005BFB05B030BD082AE4D9102A03D81B8811
:10203000ADF80830E1E7202A8DBFD3E900231B6803
:102040000293CDE90223D8E710B5CB681BB98B60AA
:102050000B618B8210BDC4681A681C60C360438A20
:10206000013B4382CA60F0E72DE9F04FD1F80080D0
:1020700093B018F0800FCDE90323C8F3C01219BF45
:10208000C8F3C03BC8F306264FF0020B1646B8F162
:10209000000F04460D4680F2D18118F0C04305932D
:1020A00040F0CC810B7B002B00F0C881BBF1020F0C
:1020B00003D00178B14240F0C48108F07F0106915D
:1020C0006AB3C8F3074A2B44069A93F8039076063E
:1020D00046EA0B4646EA82465FEAD91346EA0A0612
:1020E000079300F0908000220023CDE90A23069B8D
:1020F000009367685B4652460AA92046B847002805
:102100007ED0A7699FB9314604F10C00FFF748FB68
:102110000746E0B96FF0020013B0BDE8F08FC8F3D6
:102120000F2A18F07F0F08BF0AF0030ACBE73B69BC
:102130009E420DD03F68002FF9D1314604F10C00CA
:10214000FFF72EFB07460028E4D0A3693B60A76198
:10215000DDE90A2300264FF6FF70C6F1200E22FAB1
:1021600006F103FA0EFEA6F1200C23FA0CFC41EA5C
:102170000E0141EA0C01C9B2083609920893FFF733
:10218000E3FA402EDDE90832E7D1B882FB7D09F0A1
:102190001F06C3F384039B1BD7E9022198B2002BCF
:1021A000BCBF00F120031BB252EA0100C8F304686F
:1021B0000FD00398821A049860EB0101A74890425F
:1021C0004FF000028A4104D3079A002A5BD0012B0A
:1021D00023DDFA7D4FEA890302F0030203F07C035A
:1021E0001343FB7539462046FFF730FB079BA3B925
:1021F000FB7DC3F38402013262F38603FB7504E0C6
:102200006FF00B0088E7A76917B96FF00C0083E740
:102210003B699E42BAD03F68F6E719F0400F32D0D2
:10222000039BBB60049BFB60142200210DA8FFF7F9
:1022300033F9039B0A93049B0B932B1D0C932B7B6D
:10224000ADF83EA0013BDBB2ADF83C30069B8DF80B
:10225000433094F824308DF840B083F001038DF8BA
:1022600044308DF84160A3688DF842800AA9204669
:102270009847FB7DC3F38403013303F01F039B02E4
:10228000FB82002048E7FB7DC9F34012B2EBD31F6D
:1022900040F0DA80C3F38403B34240F0D88007995A
:1022A0002B7B4FEA9912002934D0D20741D4032B5B
:1022B00040F2D080039BBB60049BFB602B7BAE1D78
:1022C000033BDBB23246394604F10C00FFF7D0FA8B
:1022D00000280DDA20463946FFF7B8FAFB7DC3F334
:1022E0008403013303F01F039B02FB82032013E7E7
:1022F000AB883B832A7B033AB88AD2B23146FFF7D8
:1023000035FAFB7DB882DA43C2F3C01262F3C71319
:10231000FB75B6E76AB92E1D013BDBB23246394682
:1023200004F10C00FFF7A4FA0028D3DB2A7B013A62
:10233000E2E7F98AC1F30901013B0529DAB259D86C
:10234000281D002307F11A0C9A4208D910F801EB56
:102350000CF801E0013101330629DBB2F4D1039915
:102360000A9104990B91934207F11A010C9138BF1D
:10237000043379680D9134BF55FA83F300230E932B
:10238000FB8AADF83EA0C3F309031A44069B8DF8FF
:10239000433094F82430ADF83C2083F001038DF8ED
:1023A000443000238DF840B08DF841608DF84280B4
:1023B0007B602A7BB88A013A291DFFF7D7F93B8B4E
:1023C000B882834203D1A3680AA9204698472046D1
:1023D0000AA9FFF739FEFB7DB88AC3F384030133F2
:1023E00003F01F039B02FB823B8B984214BF11201A
:1023F000002091E67B68002BB1D0062001E01C3064
:102400006346D3F800C0BCF1000FF8D1091A081DCB
:1024100005F1040C00EB030905989DF8143001EB5D
:10242000000EBEF11B0F9AD89A4298D91CF8013BB6
:1024300009F8013B059B01330593EDE76FF00900B7
:102440006AE66FF00A0067E66FF00D0064E66FF071
:102450000E0061E66FF00F005EE600BF80841E0094
:10246000404BF0B51C6C404E44F000741C641D6E73
:1024700045F000751D661B6E3C4B9B6AD3F80052FD
:10248000354045F00105C3F80052D3F8004234400E
:1024900044EA002040F00100C3F80002002952D0B5
:1024A0000020C3F81C020546C3F80402C3F80C025E
:1024B000C3F8140203EBC00401301C28C4F84052D6
:1024C000C4F84452F6D100254FF0010C96781488D8
:1024D000F70748BFD3F804720CFA04F044BF07436F
:1024E000C3F80472B70742BFD3F80C720743C3F8AE
:1024F0000C72760742BFD3F814620643C3F8146225
:1025000003EBC4045668C4F840629668C4F8446299
:10251000D3F81C4201352043A942C3F81C0202F142
:102520000C02D3D1D3F8002222F00102C3F800221A
:102530000C4B1A6C22F000721A641A6E22F00072B0
:102540001A661B6EF0BD0122C3F84012C3F8441294
:10255000C3F80412C3F81412C3F80C22C3F81C22E7
:10256000E0E700BF003802400000FFFF8834002091
:10257000184A916A08B58B688B6013F0010104D08A
:1025800013F00C0F18BF4FF48031D80506D513F4A3
:10259000406F14BF41F4003141F00201D80306D569
:1025A00013F4402F14BF41F4802141F00401D3699A
:1025B0000BB108489847202383F31188064800216F
:1025C00000F0EEFD002383F31188BDE8084001F020
:1025D00017B900BF883400209034002038B5124C61
:1025E000A36ADD68AA0712D05A6922F002025A6172
:1025F000A36913B1012120469847202383F3118852
:102600000A48002100F0CCFD002383F31188EB067B
:1026100006D5A36A1021D960236A0BB102489847F6
:10262000BDE8384001F0ECB8883400209834002030
:1026300038B5124CA36A1D69AA0712D05A6922F054
:1026400010025A61A36913B1022120469847202342
:1026500083F311880A48002100F0A2FD002383F3D0
:102660001188EB0606D5A36A10211961236A0BB104
:1026700002489847BDE8384001F0C2B888340020CD
:102680009834002038B50F4CA36A5D685D602A0756
:102690000AD5042222701A6822F002021A60636AC4
:1026A00013B10021204698476B0706D5A36A9969A4
:1026B000236A13B1034809049847BDE8384001F084
:1026C0009FB800BF8834002010B50E4C204600F0A3
:1026D000CFF90D4BA3620B21132000F0B1F90B21B0
:1026E000142000F0ADF90B21152000F0A9F90B2101
:1026F000162000F0A5F90022BDE8104011460E207A
:10270000FFF7AEBE8834002000640040114B9842B1
:1027100010B5044609D1104B1A6C42F000721A64CD
:102720001A6E42F000721A661B6EA36A01221A60CA
:10273000A36A5A68D20707D5626851681268D961DE
:102740001A60064A5A6110BD0121082000F01EFCE3
:10275000EEE700BF88340020003802405B870100AC
:1027600003291AD8DFE801F0020A0F14836A9B6874
:1027700013F0E05F14BF012000207047836A98685F
:10278000C0F380607047836A9868C0F3C060704788
:10279000836A9868C0F3007070470020704700009B
:1027A00010B5032925D8DFE801F00225292D836A19
:1027B0009968C1F30161183103EB011310788406A5
:1027C0004CBF54689488C0F300114FEA410148BFE0
:1027D00041EAC40100F00F004CBF41F0040141EA9E
:1027E0004451586041F001019068D2689860DA6005
:1027F000196010BD836A03F5C073DFE7836A03F5D0
:10280000C873DBE7836A03F5D073D7E701290AD0E1
:1028100002290FD081B9836ADA68920701D1186959
:1028200003E001207047836AD86810F0030018BFE6
:1028300001207047836AF2E70020704710B539B96C
:10284000836AD96889071BD11B699C0704D110BD15
:10285000012915D00229FAD1816AD1F8C031D1F805
:10286000C441D1F8C8011061D1F8CC0150612020D9
:1028700008610869800717D1486940F0100012E02C
:10288000816AD1F8B031D1F8B441D1F8B801106102
:10289000D1F8BC0150612020C860C868800703D10E
:1028A000486940F002004861C3F34000C3F380016F
:1028B000000140EA4111107920F03000014311710C
:1028C00089064BBF91681189DB085B0D4CBF63F330
:1028D0001C0163F30A01137948BF916064F3030399
:1028E00013714FEA14234FEA144458BF1181137037
:1028F0005480ACE7024AD36843F0C003D36070470A
:1029000000440040044B5A6810439A6858600AB16A
:10291000181D1047704700BFB43400202DE9F04166
:102920003C4ED6F85C52EF682B68DA059CB20CD5A9
:10293000202383F311884FF40070FFF7E3FF6FF457
:1029400080732B60002383F31188202383F3118885
:10295000DFF8C08014F02F0339D183F311883806D3
:1029600013D5210611D5202383F311882A4800F0BE
:1029700001FA00284CDA0820FFF7C4FF4FF67F73F6
:102980003B40EB60002383F311887A0615D563067C
:1029900013D5202383F31188D6E913239A4209D152
:1029A000336C3BB127F040073F0410203F0CFFF78A
:1029B000A9FFEF60002383F31188D6F86422D3685F
:1029C0000BB110699847BDE8F04100F019BF23072B
:1029D00012D014F0080F0CBF00208020E10748BF80
:1029E00040F02000A20748BF40F04000630748BF06
:1029F00040F48070FFF786FFA4066B6805D596F853
:102A000060124046194000F057FA2C68A4B2A1E7C2
:102A10006860B7E7B4340020EC34002010B5054CF2
:102A2000054A0021204600F025FA044BC4F85C3228
:102A300010BD00BFB4340020F52800080044004059
:102A400000F1604303F561430901C9B283F8001343
:102A5000012200F01F039A4043099B0003F16043E9
:102A600003F56143C3F880211A607047FFF72CBE5D
:102A7000012300F10802C0E90222037000F11002F4
:102A80000023C0E90422C0E90633C0E908334360EB
:102A90007047000010B52023044683F311880223F9
:102AA00003704160FFF732FE04232370002383F399
:102AB000118810BD2DE9F0411F4604460D4616460B
:102AC000202383F3118800F108082378052B0DD00B
:102AD00029462046FFF744FE40B1204632462946AB
:102AE000FFF75EFE002080F3118808E0394640467B
:102AF00000F03AFB0028E8D0002383F31188BDE8FA
:102B0000F08100002DE9F0411F4604460D461646AF
:102B1000202383F3118800F110082378052B0DD0B2
:102B200029462046FFF772FE40B12046324629462C
:102B3000FFF784FE002080F3118808E03946404604
:102B400000F012FB0028E8D0002383F31188BDE8D1
:102B5000F0810000F8B5154682680669AA420B4666
:102B6000816938BF8568761AB54204460BD218468B
:102B70002A46FEF77FFCA3692B44A361A3685B1B75
:102B8000A3602846F8BD0CD918463246FEF772FC01
:102B9000AF1BE1683A463044FEF76CFCE3683B4407
:102BA000EBE718462A46FEF765FCE368E5E7000018
:102BB00083689342F7B51546044638BF8568D0E967
:102BC0000460361AB5420BD22A46FEF753FC6369FD
:102BD0002B446361A36828465B1BA36003B0F0BD70
:102BE0000DD932460191FEF745FC0199E068AF1B13
:102BF0003A463144FEF73EFCE3683B44E9E72A46A7
:102C0000FEF738FCE368E4E710B50A440024C3612A
:102C1000029B8460C0E90000C0E90511C160026147
:102C2000036210BD08B5D0E90532934201D1826834
:102C300082B98268013282605A1C42611970D0E9FF
:102C400004329A4224BFC3684361002100F09CFA19
:102C5000002008BD4FF0FF30FBE7000070B52023D7
:102C600004460E4683F31188A568A5B1A368A2693E
:102C7000013BA360531CA36115782269934224BFD2
:102C8000E368A361E3690BB120469847002383F30F
:102C90001188284607E03146204600F065FA0028F2
:102CA000E2DA85F3118870BD2DE9F74F04460E4630
:102CB00017469846D0F81C904FF0200A8AF31188E6
:102CC0004FF0000B154665B12A4631462046FFF706
:102CD00041FF034660B94146204600F045FA00280E
:102CE000F1D0002383F31188781B03B0BDE8F08F87
:102CF000B9F1000F03D001902046C847019B8BF328
:102D00001188ED1A1E448AF31188DCE7C0E9051129
:102D1000C160C3611144009B8260C0E90000016191
:102D200003627047F8B504460D461646202383F328
:102D30001188A768A7B1A368013BA36063695A1C07
:102D400062611D70D4E904329A4224BFE368636172
:102D5000E3690BB120469847002080F3118807E013
:102D60003146204600F000FA0028E2DA87F31188A5
:102D7000F8BD0000D0E905239A4210B501D1826860
:102D80007AB98268013282605A1C82611C780369B8
:102D90009A4224BFC3688361002100F0F5F9204600
:102DA00010BD4FF0FF30FBE72DE9F74F04460E460C
:102DB00017469846D0F81C904FF0200A8AF31188E5
:102DC0004FF0000B154665B12A4631462046FFF705
:102DD000EFFE034660B94146204600F0C5F90028E1
:102DE000F1D0002383F31188781B03B0BDE8F08F86
:102DF000B9F1000F03D001902046C847019B8BF327
:102E00001188ED1A1E448AF31188DCE702684368D2
:102E10001143016003B11847704700001430FFF7F9
:102E200043BF00004FF0FF331430FFF73DBF0000F9
:102E30003830FFF7B9BF00004FF0FF333830FFF7ED
:102E4000B3BF00001430FFF709BF00004FF0FF319F
:102E50001430FFF703BF00003830FFF763BF0000F6
:102E60004FF0FF323830FFF75DBF000000207047A1
:102E7000FFF7D4BD37B515460E4A02600022426006
:102E8000C0E902220122044602740B46009000F1C0
:102E90005C014FF480721430FFF7B6FE00942B46AD
:102EA0004FF4807204F5AE7104F13800FFF72EFF85
:102EB00003B030BD203F000838B5C36904460D4655
:102EC0001BB904210844FFF7A1FF294604F11400AF
:102ED000FFF7A8FE002806DA201D4FF48061BDE848
:102EE0003840FFF793BF38BD024B0022C3E90033DF
:102EF0009A6070471C370020002303748268054BDA
:102F00001B6899689142FBD25A6803604260106066
:102F1000586070471C37002008B5202383F31188C0
:102F2000037C032B05D0042B0DD02BB983F3118820
:102F300008BD436900221A604FF0FF334361FFF779
:102F4000DBFF0023F2E7D0E9003213605A60F3E7B9
:102F5000002303748268054B1B6899689142FBD873
:102F60005A68036042601060586070471C37002048
:102F7000054B19690874186802681A605360186173
:102F800001230374FDF744BB1C37002030B54B1CF4
:102F90000B4D87B0044610D02B690A4A01A800F0F7
:102FA0001BF92046FFF7E4FF049B13B101A800F0D2
:102FB0004FF92B69586907B030BDFFF7D9FFF8E723
:102FC0001C370020192F000838B50C4D41612B69C2
:102FD00081689A689142044603D8BDE83840FFF7FB
:102FE0008BBF1846FFF7B4FF01232C610146237401
:102FF0002046BDE83840FDF70BBB00BF1C37002062
:10300000044B1A681B6990689B68984294BF002023
:10301000012070471C37002010B5084C2368206938
:103020001A6822605460012223611A74FFF790FF2E
:1030300001462069BDE81040FDF7EABA1C370020C0
:1030400008B5FFF7DDFF18B1BDE80840FFF7E4BFA2
:1030500008BD0000FFF7E0BFFEE7000010B50C4C14
:10306000FFF742FF00F0AAF80A498022204600F04C
:1030700031F8012344F8180C037400F09DFB002381
:1030800083F3118862B60448BDE8104000F042B8EE
:1030900044370020483F0008583F000800F012B9AC
:1030A000EFF3118020B9EFF30583202282F311881A
:1030B0007047000010B530B9EFF30584C4F308047D
:1030C00014B180F3118810BDFFF7BAFF84F31188A3
:1030D000F9E7000082600222028270478368A3F150
:1030E0007C0243F80C2C026943F83C2C426943F8FB
:1030F000382C074A43F81C2CC26843F8102C0222D3
:1031000003F8082C002203F8072CA3F118007047DD
:103110002906000810B5202383F31188FFF7DEFF8E
:1031200000210446FFF750FF002383F31188204657
:1031300010BD0000024B1B6958610F20FFF718BF3C
:103140001C370020202383F31188FFF7F3BF000012
:1031500008B50146202383F311880820FFF716FFE6
:10316000002383F3118808BD49B1064B42681B69EF
:1031700018605A60136043600420FFF707BF4FF0E8
:10318000FF3070471C3700200368984206D01A6849
:103190000260506059611846FFF7AEBE70470000EC
:1031A00038B504460D462068844200D138BD036816
:1031B00023605C604561FFF79FFEF4E7054B03F178
:1031C0001402C3E905224FF0FF310022C3E90712C0
:1031D000704700BF1C37002070B51C4EC0E90323A8
:1031E00005460C4600F06EFB334653F8142F9A4206
:1031F0000DD13062C5E901242A600A2C2CBF0019C8
:103200000A30C6E90555BDE8704000F049BB316A97
:10321000431AE31838BF1C469368A34202D9081921
:1032200000F04CFB73699A6894420CD85A68AC6001
:103230002B606A6015609A685D60121B9A604FF09F
:10324000FF33F36170BD1B68A41AECE71C37002044
:1032500038B51B4C636998420DD0D0E90032136039
:103260005A6000228168C2609A680A449A604FF0EE
:10327000FF33E36138BD2246036842F8143F002162
:1032800093425A60C16003D1BDE8384000F010BBE2
:103290009A688168256A0A449A6000F013FB6369A2
:1032A0009A68411B8A42E5D9AB181D1A092D206A7C
:1032B00098BF01F10A02BDE83840104400F0FEBAA0
:1032C0001C3700202DE9F041184C002704F11406AA
:1032D000656900F0F7FA236AAA68C11A8A4215D80C
:1032E00013442362D5E9003213605A606369D5F84C
:1032F0000C80EF60B34201D100F0DAFA87F3118855
:103300002869C047202383F31188E1E76169B1424E
:1033100009D013441B1ABDE8F0410A2B2CBFC0187A
:103320000A3000F0CBBABDE8F08100BF1C370020A6
:1033300000207047FEE70000704700004FF0FF30AC
:1033400070470000BFF34F8F024AD368DB03FCD401
:10335000704700BF003C024008B5094B1B7873B9A9
:10336000FFF7F0FF074B1A69002ABFBF064A5A60F1
:1033700002F188325A601A6822F480621A6008BD2D
:10338000D8380020003C02402301674508B50B4BAC
:103390001B7893B9FFF7D6FF094B1A6942F0004238
:1033A0001A611A6842F480521A601A6822F4805234
:1033B0001A601A6842F480621A6008BDD83800208A
:1033C000003C02400728F0B516D80C4C0C49237875
:1033D0007BB90C4D0E4608234FF0006255F8047B74
:1033E00046F8042B013B13F0FF033A44F6D10123C6
:1033F000237051F82000F0BD0020FCE7FC380020CD
:10340000DC380020703F0008014B53F82000704763
:10341000703F000808207047072810B5044601D9FE
:10342000002010BDFFF7CEFF064B53F824301844A0
:10343000C21A0BB90120F4E712680132F0D1043B43
:10344000F6E700BF703F0008072838B5044628D8C3
:10345000FFF726FEFFF776FFFFF77EFF124AF32302
:10346000D360E300DBB243F4007343F00203136163
:10347000136943F48033136105462046FFF762FF6A
:10348000FFF7A0FF094B53F8241000F03BF9284642
:10349000FFF77CFFFFF70EFE2046BDE83840FFF740
:1034A000BBBF002038BD00BF003C0240703F000899
:1034B00012F001032DE9F04105460E4614464BD1AA
:1034C0008118334A914261D8324B1B6813F00103D3
:1034D0005CD0314FFFF7E4FDFFF73EFFF323FB60C5
:1034E000FFF730FF314640F20128032C18D824F0B2
:1034F0000104294E0C446D1A40F20118A1423369AF
:1035000005EB01072AD123F001033361FFF73EFFEA
:10351000FFF7D0FD0120BDE8F081043C0435E4E76D
:10352000AB07E4D13B6923F440733B613B6943EA59
:1035300008033B6151F8046B2E60BFF34F8FFFF718
:1035400001FF2B689E42E8D03B6923F001033B61F9
:10355000FFF71CFFFFF7AEFD0020DCE723F440730C
:103560003361336943EA080333610B883B80BFF35F
:103570004F8FFFF7E7FE3F8831F8023BBFB2BB42F7
:10358000BCD0336923F001033361E1E71846C2E799
:103590000000080800380240003C0240084908B515
:1035A0000B7828B11BB9FFF7D7FE01230B7008BDBC
:1035B000002BFCD0BDE808400870FFF7E7BE00BF55
:1035C000D838002070B582B0FFF76AFD0E4E054670
:1035D00000F078F93268904237BF0C4A0B495168C5
:1035E00014682EBFD1E9004101315160041903462E
:1035F00041F10001284601913360FFF75BFD01991D
:10360000204602B070BD00BF0039002008390020FC
:1036100070B582B0FFF744FD104E054600F052F938
:103620003268904237BF0E4A0D49516814682EBF68
:10363000D1E9004101315160041941F10001034613
:10364000284601913360FFF735FD01994FF47A72F6
:1036500000232046FCF7C4FD02B070BD00390020F5
:103660000839002010B50244064BD2B2904200D176
:1036700010BD441C00B253F8200041F8040BE0B226
:10368000F4E700BF502800400F4B30B51C6F2404F6
:1036900007D41C6F44F400741C671C6F44F400448E
:1036A0001C670A4C236843F4807323600244084B70
:1036B000D2B2904200D130BD441C00B251F8045B3C
:1036C00043F82050E0B2F4E70038024000700040B8
:1036D0005028004007B5012201A90020FFF7C2FFD2
:1036E000019803B05DF804FB13B50446FFF7F2FF41
:1036F000A04205D0012201A900200194FFF7C4FFD8
:1037000002B010BD70470000074B45F255521A60D9
:1037100002225A6040F6FF729A604CF6CC421A6060
:10372000024B01221A70704700300040143900200B
:10373000034B1B781BB1034B4AF6AA221A60704751
:103740001439002000300040034B1A681AB9034AAC
:10375000D2F874281A6070471039002000300240F7
:10376000024B4FF08072C3F874287047003002405B
:1037700008B5FFF7E9FF024B1868C0F3407008BDB9
:103780001039002008B5FFF7DFFF024B1868C0F3BF
:10379000007008BD10390020EFF3098305494A6B1A
:1037A00022F001024A63683383F30988002383F31C
:1037B0001188704700EF00E0202080F3118862B686
:1037C0000C4B0D4AD96821F4E0610904090C0A4345
:1037D000DA60D3F8FC20094942F08072C3F8FC207B
:1037E0000A6842F001020A601022DA7783F82200A8
:1037F000704700BF00ED00E00003FA05001000E094
:1038000010B5202383F311880E4B5B6813F400631B
:1038100014D0F1EE103AEFF30984683C4FF0807356
:10382000E361094BDB6B236684F30988FFF7E8FB50
:1038300010B1064BA36110BD054BFBE783F3118864
:10384000F9E700BF00ED00E000EF00E03B060008F4
:103850003E06000870470000FEE700000A4B0B48D8
:103860000B4A90420BD30B4BDA1C121AC11E22F0EA
:1038700003028B4238BF00220021FDF70DBE53F832
:10388000041B40F8041BECE79C400008983900201A
:1038900098390020983900207047000000F080B867
:1038A0004FF08043002258631A610222DA607047A9
:1038B0004FF080430022DA60704700004FF08043F1
:1038C000586370474FF08043586A70474B684360B5
:1038D0008B688360CB68C3600B6943614B6903628B
:1038E0008B6943620B6803607047000008B5234B87
:1038F00023481A6942F0FF021A611A6922F0FF0296
:103900001A611A691A6B42F0FF021A631A6D42F0CB
:10391000FF021A651B4A1B6D1146FFF7D7FF02F124
:103920001C0100F58060FFF7D1FF02F1380100F5BE
:103930008060FFF7CBFF02F1540100F58060FFF7D4
:10394000C5FF02F1700100F58060FFF7BFFF02F1D3
:103950008C0100F58060FFF7B9FF02F1A80100F5C6
:103960008060FFF7B3FF02F1C40100F58060FFF74C
:10397000ADFFBDE8084000F097B800BF0038024036
:1039800000000240903F000808B500F017FAFFF76A
:1039900065FBBDE80840FFF7D7BE00007047000098
:1039A000104B1A6C42F001021A641A6E42F00102C6
:1039B0001A660D4A1B6E936843F0010393604FF043
:1039C000804331229A624FF0FF32DA6200229A611C
:1039D0005A63DA605A6001225A6108211A601C2079
:1039E000FFF72EB800380240002004E04FF080427C
:1039F00008B51169D3680B40D9B2C9439B0711615F
:103A000007D5202383F31188FFF748FB002383F3B6
:103A1000118808BD08B5FFF7E9FFBDE80840FFF7CA
:103A2000EFBE00001E4B1A6962F0FF021A611A69AC
:103A3000D2B21A614FF0FF301A695A6958610021F9
:103A40005A6959615A691A6A62F080521A621A6A8E
:103A500002F080521A621A6A5A6A58625A6A5962A5
:103A60005A6A1A6C42F080521A641A6E42F08052FE
:103A70001A661A6E0B4A106840F480701060186F56
:103A800000F44070B0F5007F1EBF4FF4803018671F
:103A90001967536823F40073536000F06FB900BFD7
:103AA00000380240007000403B4B3C4A1A643C4ADC
:103AB0004FF4404111601A6842F001021A601A681E
:103AC0009007FCD59A6822F003029A60324B9A68FC
:103AD00012F00C02FBD1196801F0F90119609A602B
:103AE0001A6842F480321A601A689103FCD55A6F42
:103AF00042F001025A67284B5A6F9207FCD5294AB7
:103B00005A601A6842F080721A60254A5368580455
:103B1000FCD5214B1A689101FCD5234AC3F88420B7
:103B20001A6842F080621A601A681201FCD51F4AB6
:103B30009A600322C3F88C204FF00062C3F89420EF
:103B40001B4B1A681B4B9A421B4B21D11B4A116815
:103B50001B4A91421CD140F203121A60164A1368A4
:103B600003F00F03032BFAD10B4B9A6842F00202C9
:103B70009A609A6802F00C02082AFAD15A6C42F450
:103B800080425A645A6E42F480425A665B6E7047B5
:103B900040F20372E1E700BF003802400004001069
:103BA0000070004004194002083000240094883856
:103BB000002004E011640020003C024000ED00E021
:103BC00041C20F41084A08B5516913680B4003F020
:103BD0000103536123B1054A13680BB1506898473C
:103BE000BDE80840FFF70CBE003C0140183900203A
:103BF000084A08B5516913680B4003F0020353618A
:103C000023B1054A93680BB1D0689847BDE80840D6
:103C1000FFF7F6BD003C014018390020084A08B5FE
:103C2000516913680B4003F00403536123B1054A43
:103C300013690BB150699847BDE80840FFF7E0BD34
:103C4000003C014018390020084A08B55169136842
:103C50000B4003F00803536123B1054A93690BB18C
:103C6000D0699847BDE80840FFF7CABD003C014055
:103C700018390020084A08B5516913680B4003F051
:103C80001003536123B1054A136A0BB1506A984778
:103C9000BDE80840FFF7B4BD003C014018390020E2
:103CA000174B10B55A691C68144004F478725A61B5
:103CB000A30604D5134A936A0BB1D06A98476006ED
:103CC00004D5104A136B0BB1506B9847210604D5ED
:103CD0000C4A936B0BB1D06B9847E20504D5094AA7
:103CE000136C0BB1506C9847A30504D5054A936C2F
:103CF0000BB1D06C9847BDE81040FFF781BD00BF05
:103D0000003C0140183900201A4B10B55A691C6854
:103D1000144004F47C425A61620504D5164A136DBE
:103D20000BB1506D9847230504D5134A936D0BB121
:103D3000D06D9847E00404D50F4A136E0BB1506E56
:103D40009847A10404D50C4A936E0BB1D06E9847E6
:103D5000620404D5084A136F0BB1506F98472304CF
:103D600004D5054A936F0BB1D06F9847BDE810405A
:103D7000FFF746BD003C014018390020062108B578
:103D80000846FEF75DFE06210720FEF759FE0621D4
:103D90000820FEF755FE06210920FEF751FE0621F8
:103DA0000A20FEF74DFE06211720FEF749FEBDE86A
:103DB000084006212820FEF743BE000008B5FFF7A3
:103DC00031FE00F00BF8FEF751FEFFF751F8FFF758
:103DD000E5FDBDE80840FFF761BD00000023054A8E
:103DE00019460133102BC2E9001102F10802F8D183
:103DF000704700BF1839002010B5013902449042C5
:103E000001D1002005E0037811F8014FA34201D051
:103E1000181B10BD0130F2E72DE9F041A3B1C91A1A
:103E200017780144044603F1FF3C8C42204601D937
:103E3000002009E00578BD4204F10104F5D10CEB46
:103E40000405D618A54201D1BDE8F08115F8018D11
:103E500016F801EDF045F5D0E7E70000034611F84C
:103E6000012B03F8012B002AF9D170476F72672EDE
:103E70006172647570696C6F742E41524B5F47506C
:103E8000530000004E6F20617070207369670A0054
:103E9000426164206677206C656E677468202575C2
:103EA0000A0042616420626F6172645F6964202568
:103EB000752073686F756C642062652025750A0033
:103EC0004261642066772064657363726970746F01
:103ED00072206C656E6774682025750A0042616403
:103EE0002061707020435243203078253038783A72
:103EF000307825303878203078253038783A307866
:103F0000253038780A00476F6F64206669726D77D4
:103F10006172650A0040A2E4F16468910600000045
:103F200000000000392E0008252E0008612E000830
:103F30004D2E0008592E0008452E0008312E00088D
:103F40001D2E00086D2E00086D61696E00000000D6
:103F500069646C6500000000503F00086037002075
:103F6000D83800200100000059300008000000008F
:103F70000040000000400000004000000040000041
:103F8000000001000000020000000200000002002A
:103F9000A000902A00000000AAAAAAAA50000024AB
:103FA000FFFB000000770000009009000100000501
:103FB00000000000AAAAAAA501000080FFEF0000EF
:103FC00000000000000000000000000000000000F1
:103FD000AAAAAAAA00000000FFFF0000000000003B
:103FE000000000000000000000000000AAAAAAAA29
:103FF00000000000FFFF00000000000000000000C3
:104000000000000000000000AAAAAAAA0000000008
:10401000FFFF0000000000000000000000000000A2
:1040200000000000AAAAAAAA00000000FFFF0000EA
:104030000000000000000000000000000000000080
:10404000AAAAAAAA00000000FFFF000000000000CA
:104050000000000000000000000000000A00000056
:10406000000000000300000000000000000000004D
:10407000A0C1FF7F0100000051000000000000000F
:1040800000000700000000006400000000000000C5
:0C40900040420F00FE2A0100D204000094
:00000001FF
